:020000040000FA
:10000000B201E72AA9008030A0008430A1001E3090
:10001000A400A501A722AA012108031916282A1461
:100020005220FC3E031C1628AA1452202003AB00C9
:10003000280F1E28FF30A400A50029282808A500A5
:10004000A401A600A7012B0A03192928A200A301D5
:10005000C122A90B42281708CF39A41B2038241B22
:1000600010380C3897002508950083160711831265
:100070002B088316920083121208FC392A040438D4
:100080009200E22AA90B51281D08CF39A41B203861
:10009000241B10380C389D0025089B008316871000
:1000A0003728E22AA10CA00CA10CA00C0800B21663
:1000B000B21EB212B2196028B2159920031887280F
:1000C0000830A300AD20A20DA30B6228B21E92201F
:1000D000B720B320B21A87208C2022080310E22A0E
:1000E000B216B21EB21232197A28FE39B300321596
:1000F0000310E22A321A8228A60032169920031829
:1001000087282608A02003188728B21EE22A9220FA
:10011000B72032113212B211360884003408841725
:1001200080049828360884003409800584178005E7
:1001300008008C20B7209220B3203308B219013870
:10014000A2000830A300A20D03188C20031C9220EB
:10015000B720B320A30BA3288C20B7203608840037
:1001600034080005FF3E3708840035099528370814
:10017000840035088F28A501A400B3172730A300F9
:100180001030CE200330A300E830CE20A30164302D
:10019000CE20A3010A30CE202408D928A2002508A9
:1001A000A1002408A000A5222008031DB313B31B3F
:1001B0000800303EDC280408A7008710071007104D
:1001C0008316871007100710860183122708B218BC
:1001D00004293A30A100FC3053223330A600172105
:1001E0001030A100683053221721643052221721A9
:1001F000383003210C300321013003210630032164
:10020000B214270804293214A600321C1229071040
:10021000033C031C172917210730A100D0305322BB
:10022000031408003214FE3C0319E22A0714871451
:10023000260886003210871032305222031408003C
:100240002C08A0002D08A1000130A200A301640029
:100250004E21031C3B29A20B2729FF30A3070318BB
:100260002729A007031CA107031C08006430A20073
:100270000030A3002729AB21A8010830A300AC213E
:100280004E210318A80AAB1EA801A20CA30B3F29FC
:10029000AB1AA213AC21031422080800360884000C
:1002A000340884178004841300052B1B3406FF3E9A
:1002B0000800290803140319E22ADD22031C0800A0
:1002C000A9035929A400290803140319E22ADD22ED
:1002D000031C0800A00025188317240884002008A8
:1002E00080008313A40AA90363290408A600360822
:1002F00084008030B3050830A70003100318B30A48
:100300009121A60CA70B7E290000AB1A330C91217A
:10031000E522031491212F08A3002E08462203147E
:10032000E22A8413AB1FA029000834042B1F3406D3
:100330008000841700083404031C34068000AC29B4
:1003400000083404031C34062B1B34068000841779
:1003500034098005AC2933172B081F39003EA10052
:100360002A08043E0318A10A331F532A3313A0009E
:100370000310A10CA00C0310A10C200C532AB313E2
:1003800029080319B3171030A8000301A40DA50D07
:1003900003180130FF212808031DC5290800B313E5
:1003A00029080319B3170430A800250EDC212508FD
:1003B000DC21240EDC2124080F39F63E0318073E09
:1003C0000A3EFF29B31329080319B3170530A80003
:1003D0002730A3001030F8210330A300E830F821C3
:1003E000A3016430F821A3010A30F8212408FF2971
:1003F000A2002508A1002408A000A5222008A00032
:10040000A8030319B31329080319092A280203189A
:1004100008002008031DB313B31B0800303EDD2A7B
:100420000F39A0000310A00DA00D1F08C039200433
:1004300001389F000030A100323053229F149F18D2
:100440001F2AA1011E08E22A83178001840AFF3EA9
:10045000031D252AE22A031783168C010C1483122C
:100460000C0803178D0AE22A030103178C00831678
:100470008C010C1555308D00AA308D008C148C1811
:100480003F2A0C1183128D0AE22AA301A200FF3039
:10049000A207031CA307031CE22A0330A100E330D8
:1004A0005322472AA101F43EA000A109FE30031CFB
:1004B0005C2AA0070318592AA0076400A10F592A33
:1004C00000002018632A2018652A0800A000A11B3C
:1004D000D7222008E22A0310A10CA00CFF3E03182B
:1004E0006B2A2008E22AA2000330802AA101A3017E
:1004F000A2000130802AA101A301A2000430802AB9
:10050000A80023082102031D872A220820020430A4
:1005100003180130031902302805031DFF30E22AB9
:100520000038031DFF300405031DFF30E22AA2003E
:100530002008A6002408A0002608A4002108A60080
:100540002508A1002608A500A72AA501A4011030AE
:10055000A600210DA40DA50D2208A4022308031C4A
:10056000230FA5020318BB2A2208A4072308031897
:10057000230FA5070310A00DA10DA60BA92A200883
:10058000E22A1030A800A101A001A70CA60C031CB0
:10059000CF2A2208A00723080318230FA107A10CC4
:1005A000A00CA50CA40CA80BC52A2408E22AA009BB
:1005B000A109A00A0319A10A0800840031088A00D1
:1005C0003008820083130313831264000800C030D4
:1005D0009F00831675308F008312031787018801EF
:1005E00003133030900083160B3085008601903065
:1005F00087000317013088008901831203138130BB
:100600009F0083169F018312051283160512831221
:100610000511831605118312851283168512831224
:10062000871283168712831285138316851383120C
:1006300005178316051320308400603083128A0169
:100640002522A030840050308A01252210308400F9
:1006500060308A0124229030840060308A01242294
:1006600003178D0103138A012B228316A400831222
:100670008A012B228316A50083128A012B2283165E
:10068000A60083128A012B228316A70083128A01F7
:100690002B22E6008A012B22E7008A012B22E800A8
:1006A0008A012B22E9008A012B22EC008A012B22ED
:1006B000ED008A012B228316D80083128A012B2297
:1006C0008316DE0083128A012B228316B800831260
:1006D0008A012B228316B40083120317EE308D009B
:1006E00003138A012B22D7008A012B22D8008A010A
:1006F0002B22D9008A012B22DA008A012B22D20078
:100700008A012B22D3008A012B22D4008A012B22BA
:10071000D5000317F6308D0003138A012B228316B0
:10072000D10083128A012B228316D00083128A0102
:100730002B228316C80083128A012B228316C9003C
:1007400083128A012B228316CA0083128A012B226C
:100750008316CB0083128A012B228316CC008312CE
:100760008A012B228316CD0083128A012B22831645
:10077000CE0083128A012B228316CF003808831201
:10078000A800F430A2000130A30001308A01022049
:100790000630A300D6308A01462283165108831200
:1007A0008A01DC208316500883128A01DC2057302E
:1007B0008A01DC2041308A01DC2049308A01DC20BA
:1007C00054308A01DC2049308A01DC204E308A0115
:1007D000DC2047308A01DC2020308A01DC204630D2
:1007E0008A01DC204F308A01DC2052308A01DC2073
:1007F00020308A01DC204F308A01DC2042308A011F
:10080000DC2044308A01DC2020308A01DC2050309A
:100810008A01DC204F308A01DC2052308A01DC2042
:1008200054308A01DC208A150A16352564008316A7
:100830004708003C8A110A1683120319C3280516BB
:1008400083160512C83083128A01452205128316C9
:10085000051283120130A30090308A01462205164A
:100860008316051283120130A30090308A014622BC
:1008700005128316051283120130A30090308A01FD
:10088000462205168316051283120130A30090300C
:100890008A01462205128316051283120130A30035
:1008A00090308A0146220530B6001030B4004C303A
:1008B000AA004030AB00AE01AF01F7308A017621CB
:1008C0000530B6000830B4004C30AA00AB016430EB
:1008D000AC00AD018A0120218A110A12031CC82B29
:1008E0008316BE0064003E08CC3C8A110A128312B3
:1008F000031D042B8316510883128A01DC20831602
:10090000500883128A01DC20DC30F6000B30F7003F
:10091000101076088E0077088F000C1010146400F9
:100920008A110A128518012D8316510883128A0133
:10093000DC2008308A01DC20A801F430A20001305C
:10094000A30001308A0102208513831685138312C8
:1009500087128316871283128512831685128312DB
:1009600003178D0183160313240883128A0135228D
:100970008316250883128A013522831626088312DE
:100980008A0135228316270883128A0135226608D8
:100990008A01352267088A01352268088A013522D2
:1009A00069088A0135226C088A0135226D088A019E
:1009B00035228316580883128A01352283165E0871
:1009C00083128A0135228316380883128A01352260
:1009D0008316340883128A0135223A30A3009830F6
:1009E0008A01462264008A110A12851CF22C8316A1
:1009F000510883128A01DC200C308A01DC208A0134
:100A0000042B8A150A163525640083164708003C16
:100A10008A110A1683120319C32864008316470833
:100A2000013C8A110A1683120319CA2F6400831627
:100A30004708023C8A110A1683120319172E640014
:100A400083164708033C8A150A16831203196C297A
:100A5000640083164708043C8A150A12831203199E
:100A6000B42E8316BE0183128A110A127A268316C7
:100A7000510883128A01DC208316480883128A01F8
:100A8000DC208A150A12112183160130BE0051089C
:100A900083128A01DC208316490883128A01DC2034
:100AA0008A150A12112183160230BE0051088312E2
:100AB0008A01DC2083164A0883128A01DC208A1509
:100AC0000A12112183160330BE00510883128A01D5
:100AD000DC2083164B0883128A01DC208A150A1257
:100AE00011218316BE01510883128A01DC2083166E
:100AF0004C0883128A01DC208A150A1215238A15F4
:100B00000A1265268316BE0183128A110A127A26FA
:100B10008316510883128A01DC2083164808831249
:100B20008A01DC208A150A12112183160130BE00C9
:100B3000510883128A01DC208316490883128A0136
:100B4000DC208A150A12112183160230BE005108DA
:100B500083128A01DC2083164A0883128A01DC2072
:100B60008A150A12112183160330BE005108831220
:100B70008A01DC2083164B0883128A01DC208A1547
:100B80000A12112183160130BE00510883128A0116
:100B9000DC2083164D0883128A01DC208A150A1294
:100BA00015238A150A1265268316BE0183128A113F
:100BB0000A127A268316510883128A01DC208316D2
:100BC000480883128A01DC208A150A121121831633
:100BD0000130BE00510883128A01DC2083164908C7
:100BE00083128A01DC208A150A1211218316023031
:100BF000BE00510883128A01DC2083164A08831242
:100C00008A01DC208A150A12112183160330BE00E6
:100C1000510883128A01DC2083164B0883128A0153
:100C2000DC208A150A12112183160230BE005108F9
:100C300083128A01DC2083164E0883128A01DC208D
:100C40008A150A1215238A150A1265268316BE0113
:100C500083128A110A127A268316510883128A0196
:100C6000DC208316480883128A01DC208A150A12C8
:100C7000112183160130BE00510883128A01DC2045
:100C80008316490883128A01DC208A150A12112171
:100C900083160230BE00510883128A01DC208316BD
:100CA0004A0883128A01DC208A150A121121831650
:100CB0000330BE00510883128A01DC2083164B08E2
:100CC00083128A01DC208A150A121121831603304F
:100CD000BE00510883128A01DC2083164F0883125C
:100CE0008A01DC208A150A1215238A150A12652644
:100CF0008A018F2C83163C1405308312B600043011
:100D0000B4005430AA004030AB00AE01AF01E43073
:100D10008A01762106308A01762102308A01762105
:100D20000B308A01762110308A017621F9308A0150
:100D300076210530B6000230B4005430AA00AB0171
:100D40006430AC00AD010330A9002030B0000130A8
:100D5000B1008A0159218A110A12031CC02E1030D9
:100D6000A9002030B0000130B100A50138308A015F
:100D700062218A110A12031CC02E83163C108312B2
:100D800064008A110A12831683103C1C8314831298
:100D90008318CB2E08000B3038078316B30083125C
:100DA0003D08FB003E08FA003F088316B00083129E
:100DB0003F08E1004008E00064008A110A1283162F
:100DC0008310B01F831483128318ED2E83162B30EB
:100DD000B00083128A110A12F12E83162D30B00052
:100DE00083126108A10060088A016622E0002108E0
:100DF000E1006008A6006108A700E830A200033007
:100E0000A3008A01C122E0002508E100A301CD3042
:100E10008A019722E0002108E10064008A110A1289
:100E200083168310B4198314831283182A2F600841
:100E3000A6006108A7009330A200A3018A01C12285
:100E4000E0002508E100A30164308A019722E00058
:100E50002108E10042084307FE00FF01FF0D7F0C5F
:100E60007E0C8316E10064001E3061028A110A12B2
:100E700083120318452F831661081E3CE1002D30B4
:100E8000E20083128A110A124B2F1E308316E102F0
:100E90002B30E200831264008A110A128316831039
:100EA0003419831483128318582F8A150A16FE25C5
:100EB00083166108E000831245088316C1000430E0
:100EC000831246078316B10083126008A0006108F0
:100ED000A1006430A200A3018A01A522FE0021081E
:100EE000FF00831633088312A600A7017E08A20024
:100EF0007F08A3008A01C1228316AC008312250853
:100F00008316AD0083126008A0006108A100A30150
:100F100064308A0173228A110A12031D932F8316EB
:100F20003308DA0083126400831630082B3C8A11E0
:100F30000A128312031DE02F83162C08A8072D0820
:100F40000318013EA9078312831628088312A00004
:100F5000831629088312A1003830A30040308A018B
:100F60007D228A110A12031DC22F8316A40A0319B7
:100F7000A50A4030A8023830031C013EA9028312A2
:100F80008A01A42F6008E40761080318013EE50701
:100F90006408A0006508A1003830A30040308A0131
:100FA0007D228A110A12031DE02FE60A0319E70ABF
:100FB0004030E4023830031C013EE5028A01C82FAC
:100FC0006400831630082D3C8A150A128312031D13
:100FD0007C286008A0006108A1006430A200A30181
:100FE0008A01A5228316B50035088312A0001830A7
:100FF0008A017622FE00831635088312A000243071
:101000008A017B228316A00083127E088400831647
:10101000200883128A0190228316A000A100640098
:10102000200821048A150A12831203193628831610
:1010300033085A02E60066088312A600A701E830CA
:10104000A2000330A3008A01C122FE002508FF0090
:101050007E08A0007F08A100831635088312A20035
:10106000A3018A01A522E2002108E30083162C08CF
:10107000AA072D080318013EAB07831283162A081E
:101080008312A00083162B088312A1003830A3001E
:1010900040308A017D228A150A12031D5D288316BD
:1010A000A60A0319A70A4030AA023830031C013EE1
:1010B000AB0283128A150A123E286008EA0761080B
:1010C0000318013EEB076A08A0006B08A100383046
:1010D000A30040308A017D228A150A12031D7C2854
:1010E000E80A0319E90A4030EA023830031C013EDD
:1010F000EB028A150A12632864008A150A12831605
:101100008310B41F83148312831810290730B6008C
:101110004030B4005430AA004030AB00AE01AF0103
:1011200044308A01762141308A01762154308A0187
:10113000762141308A0176212C308A017621543083
:101140008A01762149308A0176214D308A01762143
:1011500045308A0176212C308A017621A901831637
:1011600033088312A400A5017530B0000130B1002E
:101170008A01E2212C308A017621831630088312FD
:101180008A0176212C308A017621A9016008A40009
:101190006108A5007530B0000130B1008A01E2217C
:1011A0002C308A017621A9017A08A4007B08A500C9
:1011B0007530B0000130B1008A01E2212C308A0183
:1011C0007621A901831660088312A400A501753059
:1011D000B0000130B1008A01E2212C308A01762171
:1011E000A90183162C088312A40083162D088312EC
:1011F000A5007530B0000130B1008A01E2212C3029
:101200008A017621A9016208A4006308A50075304F
:10121000B0000130B1008A01E2210D308A0176214F
:10122000080083163E08523E840083120008FE0028
:1012300064007E080B3C8A150A12031D33295630C0
:101240008A01DC204F308A01DC204C308A01DC200E
:1012500020308A01DC208316330883128A01BB20E8
:1012600020308A01DC2083163E08523E840083121F
:101270000008FE0064007E08103C8A150A12031D57
:10128000792953308A01DC204F308A01DC20433039
:101290008A01DC2020308A01DC207A08A0007B084B
:1012A000A1000A30A200A3018A01A522FE002108A4
:1012B000FF007F08A5007E088A01BC202E308A012D
:1012C000DC207A08A0007B08A1000A30A200A3015C
:1012D0008A01A5222408FE002508FF007F08A5003A
:1012E0007E088A01BC2020308A01DC2020308A015F
:1012F000DC2083163E08523E840083120008FE0064
:1013000064007E08123C8A150A12031DCD29413063
:101310008A01DC204D308A01DC2050308A01DC203B
:101320008316300883128A01DC206008A00061085F
:10133000A1006430A200A3018A01A522FE002108B9
:10134000FF007F08A5007E088A01BC202E308A019C
:10135000DC206008A0006108A1006430A200A301A5
:101360008A01A5222408FE002508FF007E08A000AF
:101370007F08A1000A30A200A3018A01A522FE0075
:101380002108FF007F08A5007E088A01BC202030CC
:101390008A01DC2020308A01DC2083163E08523E80
:1013A000840083120008FE0064007E08153C8A1544
:1013B0000A12031DF12954308A01DC2045308A01CC
:1013C000DC204D308A01DC208316620883128A01FA
:1013D000DC208316600883128A01BB2020308A013A
:1013E000DC2083163E08523E840083120008FE0073
:1013F00064007E08FC3C8A150A12031D162A493037
:101400008A01DC204E308A01DC204B308A01DC204E
:1014100020308A01DC208316410883128A01BB2018
:1014200030308A01DC2020308A01DC2083163E081F
:10143000523E840083120008FE0064007E08FD3CDA
:101440008A150A12031D5B2A31308A01DC203230F2
:101450008A01DC2056308A01DC2020308A01DC2021
:10146000831631088312A000A1010A30A200A30153
:101470008A01A522FE002108FF007F08A5007E0842
:101480008A01BC202E308A01DC20831631088312A9
:10149000A000A1010A30A200A3018A01A52224080C
:1014A000FE002508FF007F08A5007E088A01BC20F9
:1014B00020308A01DC2083163E08523E84008312CD
:1014C0000008FE0064007E08FE3C8A150A12031D17
:1014D000BB2A49308A01DC204E308A01DC205230A0
:1014E0008A01DC2020308A01DC206208A000630829
:1014F000A100E830A2000330A3008A01A522FE006B
:101500002108FF007F08A5007E088A01BC202E303C
:101510008A01DC206208A0006308A100E830A20074
:101520000330A3008A01A5222408FE002508FF003D
:101530007E08A0007F08A1000A30A200A3018A0152
:10154000A522FC002108FD007C08A0007D08A10068
:10155000A3010A308A0173228A150A12031DB32AD5
:1015600030308A01DC207D08A5007C088A01BC207F
:1015700020308A01DC2083163E08523E840083120C
:101580000008FE0064007E08FF3C8A150A12031D55
:10159000142B57308A01DC2041308A01DC20543082
:1015A0008A01DC2020308A01DC2083162C0883127B
:1015B000A00083162D088312A100E830A20003309A
:1015C000A3008A01A522FE002108FF007F08A500D4
:1015D0007E088A01BC202E308A01DC2083162C086C
:1015E0008312A00083162D088312A100E830A20008
:1015F0000330A3008A01A5222408FE002508FF006D
:101600007E08A0007F08A1006430A200A3018A0127
:10161000A522FE002108FF007F08A5007E088A01A0
:10162000BC2020308A01DC20080083163E08573E8B
:10163000840083120008FE006400FA307E028A15DE
:101640000A1203180A2E83163C143E08573E8400E3
:1016500083120008FE00C4307E078316C6000530E2
:101660008312B6001030B4004C30AA004030AB00FA
:10167000AE01AF0168308A0176216A308A01762195
:10168000F1308A01762101308A01762183163E08E5
:10169000573E840083120008FE007E088A017621EE
:1016A0008316460883128A0176210530B600083079
:1016B000B4004C30AA00AB016430AC00AD0107307F
:1016C000A9002030B0000130B100A50138308A01F6
:1016D00062218A150A12031C702B83163C10831298
:1016E00064008A150A12831683103C1C831483122B
:1016F00083187B2B080083163E08573E8400831214
:101700000008FE0064007E08043C8A150A12031DCE
:10171000B72B3D08A600A7016430A200A3018A01EF
:10172000C122FE002508FF007E08A0007F08A1005E
:10173000FF30A200A3018A01A5228316D2004C30FB
:1017400083128A01DC204F308A01DC2044308A0178
:10175000DC2020308A01DC208316520883128A01A3
:10176000BB2020308A01DC2020308A01DC20831657
:101770003E08573E840083120008FE0064007E0885
:10178000053C8A150A12031D2D2C640028303D02E9
:101790008A150A120318D62B3D08283C8316E1004F
:1017A0002D30E20083128A150A12DD2B28303D020B
:1017B0008316E1002B30E200831264006A30831646
:1017C00061028A150A128312031CFB2B64008A151E
:1017D0000A1283168310341F831483128318F42B88
:1017E0008517831685138312871683168712831233
:1017F0008A150A12032C8513831685138312871208
:1018000083168712831264008A150A1283168310C6
:101810003419831483128318102C8A150A16FE2596
:1018200083166108BB00453083128A01DC204330F7
:101830008A01DC2054308A01DC208316620883127E
:101840008A01DC2083163B0883128A01BB202030EA
:101850008A01DC2020308A01DC2083163E08573EB6
:10186000840083120008FE0064007E080B3C8A1589
:101870000A12031D532C3D088316D4004D308312E9
:101880008A01DC2041308A01DC2050308A01DC20D2
:1018900020308A01DC208316540883128A01BB2081
:1018A00020308A01DC2083163E08573E84008312D4
:1018B0000008FE0064007E080C3C8A150A12031D15
:1018C000932C3D08A600A701A2010130A3008A01C4
:1018D000C122FE002508FF003E08FE070318FF0A8C
:1018E0007E08A0007F08A1000430A200A3018A01A5
:1018F000A522F8002108F90052308A01DC2050307E
:101900008A01DC204D308A01DC2020308A01DC2075
:101910007908A50078088A01BC2020308A01DC20E3
:1019200020308A01DC2083163E08573E8400831253
:101930000008FE0064007E080D3C8A150A12031D93
:10194000EE2C3D088316DD0064008A150A12831010
:10195000341C831483128318DA2C83165D088312D7
:10196000A600A7014530A2001830A3008A01C122B9
:101970008316DD0083122730A30010308A019722DE
:101980008316DD004D3083128A01DC2050308A013D
:10199000DC2048308A01DC2020308A01DC208316DC
:1019A0005D0883128A01BB2020308A01DC208A1561
:1019B0000A12EE2C4B308A01DC204D308A01DC20EB
:1019C00048308A01DC2020308A01DC2083165D0843
:1019D00083128A01BB2020308A01DC2083163E0856
:1019E000573E840083120008FE0064007E080E3C0F
:1019F0008A150A12031D192D03103D0CFE00FF016C
:101A000040307E028316C400493083128A01DC20F4
:101A100047308A01DC204E308A01DC2020308A01E8
:101A2000DC208316440883128A01BB2020308A01FF
:101A3000DC2083163E08573E840083120008FE0017
:101A400064007E080F3C8A150A12031D692D64008C
:101A500028303D028A150A120318382D3D08283C0B
:101A60008316E1002D30E20083128A150A123F2D01
:101A700028303D028316E1002B30E200831264001F
:101A80008A150A128316831034198314831283185B
:101A90004C2D8A150A16FE2583166108AF004930C1
:101AA00083128A01DC2041308A01DC2054308A0113
:101AB000DC208316620883128A01DC2083162F083B
:101AC00083128A01BB2020308A01DC2020308A0169
:101AD000DC2083163E08573E840083120008FE0077
:101AE00064007E08113C8A150A12031DA22D3D08D0
:101AF000A600A7016430A200A3018A01C122FE0052
:101B00002508FF007E08A0007F08A100FF30A2008A
:101B1000A3018A01A5228316E300543083128A01AF
:101B2000DC2050308A01DC2053308A01DC20203058
:101B30008A01DC208316630883128A01BB202030CF
:101B40008A01DC2083163E08573E84008312000879
:101B5000FE0064007E08143C8A150A12031DCC2D79
:101B600003103D0C8316AE004F3083128A01DC2037
:101B700032308A01DC2031308A01DC2020308A01B9
:101B8000DC2083162E0883128A01BB2020308A01B4
:101B9000DC2020308A01DC2083163E08573E84007A
:101BA00083120008FE0064007E08153C8A150A12A4
:101BB000031D0A2E03103D0C8316DB004F308312E9
:101BC0008A01DC2032308A01DC2032308A01DC20BC
:101BD00020308A01DC2083165B0883128A01BB2037
:101BE00020308A01DC2020308A01DC20640083164A
:101BF0005B08003C8A150A128312031D062E851607
:101C00008316851283128A150A120A2E85128316EC
:101C10008512831283163E08573E84008312000803
:101C2000FE0064007E08FE3C8A150A12031D372E52
:101C300083160630C30083128A150A169B25720884
:101C4000DE007308DF004D308A01DC2045308A0158
:101C5000DC2041308A01DC2020308A01DC205F0852
:101C6000A5005E088A01BC2020308A01DC20831692
:101C70003E08573E840083120008FE0064007E0880
:101C8000FF3C8A150A12031D642E83160730C30019
:101C900083128A150A169B257208F4007308F50052
:101CA0004D308A01DC2045308A01DC204F308A012A
:101CB000DC2020308A01DC207508A50074088A0128
:101CC000BC2020308A01DC2008000F088316A30006
:101CD00083120E088316A200831264008A150A126A
:101CE0000C1C6D2E8316E40A64006408043C8A15FB
:101CF0000A128312031D982E8316E401DE0A640083
:101D00003C305E028A150A128312031C982E831639
:101D1000DE01D80A64003C3058028A150A12831288
:101D2000031C982E8316D8018312EC0A0319ED0ABE
:101D300010100F088316A30083120E088316A2004A
:101D4000831276088316A207831277080318013ED0
:101D50008316A307230883128F0083162208831299
:101D60008E000C10101408008316510883128A018B
:101D7000DC208316500883128A01DC2044308A015B
:101D8000DC2069308A01DC2073308A01DC2070306D
:101D90008A01DC206C308A01DC2061308A01DC2081
:101DA00079308A01DC2020308A01DC2053308A011E
:101DB000DC2065308A01DC206C308A01DC20653053
:101DC0008A01DC2063308A01DC2074308A01DC2047
:101DD0000730A300D0308A0146228316B501831252
:101DE0008316510883128A01DC2083164808831267
:101DF0008A01DC2049308A01DC206D308A01DC2038
:101E000061308A01DC2020308A01DC200230A90008
:101E10005208A400A501DB30B000B1018A01CF2136
:101E200020308A01DC2020308A01DC204F308A01FA
:101E3000DC2062308A01DC2064308A01DC20203022
:101E40008A01DC200230A9005708A400A501DB307C
:101E5000B000B1018A01CF2120308A01DC2020307E
:101E60008A01DC2064000130831635028A150A12CB
:101E70008312031C7D2F8316510883128A01DC20F4
:101E80008316490883128A01DC2049308A01DC204C
:101E90006D308A01DC2061308A01DC2020308A012B
:101EA000DC200230A9005308A400A501DB30B000FB
:101EB000B1018A01CF2120308A01DC2020308A0143
:101EC000DC204F308A01DC2062308A01DC20643063
:101ED0008A01DC2020308A01DC200230A900580869
:101EE000A400A501DB30B000B1018A01CF21203070
:101EF0008A01DC2020308A01DC2064000230831655
:101F000035028A150A128312031CC82F8316510842
:101F100083128A01DC2083164A0883128A01DC209E
:101F200049308A01DC206D308A01DC2061308A0171
:101F3000DC2020308A01DC200230A9005408A400F3
:101F4000A501DB30B000B1018A01CF2120308A0128
:101F5000DC2020308A01DC204F308A01DC20623016
:101F60008A01DC2064308A01DC2020308A01DC20F8
:101F70000230A9005908A400A501DB30B000B1016E
:101F80008A01CF2120308A01DC2020308A01DC2028
:101F900064000330831635028A110A168312031C6B
:101FA00013288316510883128A01DC2083164B08FC
:101FB00083128A01DC2049308A01DC206D308A01DD
:101FC000DC2061308A01DC2020308A01DC200230F4
:101FD000A9005508A400A501DB30B000B1018A01B9
:101FE000CF2120308A01DC2020308A01DC204F30D4
:101FF0008A01DC2062308A01DC2064308A01DC2026
:1020000020308A01DC200230A9005A08A400A50172
:10201000DB30B000B1018A01CF2120308A01DC2001
:1020200020308A01DC200130A300F4308A014622EE
:102030008A150A163525640083164708003C8A1164
:102040000A168312031D4C288316B50A640035084E
:10205000043C8A110A168312031D4C280317EE3024
:102060008D00031357088A01352258088A0135224A
:1020700059088A0135225A088A01352252088A01F4
:10208000352253088A01352254088A013522550821
:102090008A0135228A01C82B640083164708013C57
:1020A0008A110A168312031D682883163508523ECA
:1020B000840083120008FE0001307E07FE00FF014D
:1020C000FF0D83163508523E840083127E0880007F
:1020D000640083164708023C8A110A168312031D06
:1020E000842883163508573E840083120008FE00BA
:1020F00001307E07FE00FF01FF0D83163508573EB5
:10210000840083127E088000640083164708033C25
:102110008A110A168312031DA22883163508523E1F
:10212000840083120008FE00FF307E07FE00FF30AF
:102130000318013EFF0083163508523E84008312C7
:102140007E088000640083164708043C8A110A1642
:102150008312031DC02883163508573E840083125E
:102160000008FE00FF307E07FE00FF300318013E2E
:10217000FF0083163508573E840083127E088000D6
:102180008A150A12F02E8316510883128A01DC2068
:102190008316500883128A01DC204F308A01DC202C
:1021A00042308A01DC2044308A01DC2049308A0137
:1021B000DC2049308A01DC2043308A01DC202630D3
:1021C0008A01DC2043308A01DC2020308A01DC20B7
:1021D00056308A01DC2030308A01DC202E308A0122
:1021E000DC2030308A01DC2032308A01DC2083168A
:1021F000510883128A01DC208316490883128A0160
:10220000DC2055308A01DC203D308A01DC2053304F
:102210008A01DC2063308A01DC2073308A01DC20F3
:1022200020308A01DC204D308A01DC206F308A01A9
:10223000DC2064308A01DC2065308A01DC2020301B
:102240008A01DC2044308A01DC203D308A01DC2018
:1022500054308A01DC2065308A01DC206D308A012F
:10226000DC2070308A01DC2043308A01DC202F30F2
:102270008A01DC2046308A01DC2083165108831253
:102280008A01DC2083164A0883128A01DC2052303E
:102290008A01DC203D308A01DC2041308A01DC20CB
:1022A0006D308A01DC2070308A01DC2073308A01B5
:1022B000DC202B308A01DC2033308A01DC203230F4
:1022C0008A01DC2025308A01DC2020308A01DC20D4
:1022D0004C308A01DC203D308A01DC204D308A01FF
:1022E000DC2070308A01DC2068308A01DC202F304D
:1022F0008A01DC204B308A01DC206D308A01DC2031
:1023000068308A01DC200330A300E8308A014622CD
:102310008316510883128A01DC2083164B0883122E
:102320008A01DC2043308A01DC206F308A01DC2006
:102330006E308A01DC2066308A01DC2069308A0137
:10234000DC2067308A01DC2020308A01DC203D302F
:102350008A01DC2020308A01DC200230A9008316AB
:1023600034088312A400A501DB30B000B1018A015A
:10237000CF2120308A01DC200830A90083163408E0
:102380008312A400A501DB30B000B1018A01BF2196
:102390000130A300F4308A0146228A150A16352539
:1023A000640083164708003C8A110A168312031939
:1023B000242A640083164708013C8A110A168312F6
:1023C000031DEB2983160301B41C013E0319B4104D
:1023D000031DB4148312640083164708023C8A115B
:1023E0000A168312031DFD2983160301B41D013E45
:1023F0000319B411031DB415831264008316470832
:10240000033C8A110A168312031D0F2A8316030147
:10241000341D013E03193411031D34158312640069
:1024200083164708043C8A110A168312031D212AC9
:1024300083160301341C013E03193410031D3414A8
:1024400083128A110A1688298316510883128A0179
:10245000DC208316500883128A01DC2055308A0163
:10246000DC203D308A01DC2042308A01DC206530EE
:102470008A01DC2065308A01DC2070308A01DC2092
:1024800020308A01DC2044308A01DC203D308A0182
:10249000DC2041308A01DC206C308A01DC20613094
:1024A0008A01DC2072308A01DC206D308A01DC2058
:1024B0008316510883128A01DC208316490883128F
:1024C0008A01DC2052308A01DC203D308A01DC2088
:1024D0004C308A01DC206F308A01DC2067308A01B1
:1024E000DC2067308A01DC2069308A01DC206E3014
:1024F0008A01DC2067308A01DC2020308A01DC2060
:102500004C308A01DC203D308A01DC2056308A01C3
:10251000DC206F308A01DC206C308A01DC207430D2
:102520008A01DC2073308A01DC202D308A01DC2016
:1025300031308A01DC2035308A01DC200330A300F1
:10254000E8308A0146228316510883128A01DC2072
:1025500083164B0883128A01DC2043308A01DC2079
:102560006F308A01DC206E308A01DC2066308A01FF
:10257000DC2069308A01DC2067308A01DC202030D1
:102580008A01DC203D308A01DC2020308A01DC20F9
:102590000230A900831634088312A400A501DB30A1
:1025A000B000B1018A01CF2120308A01DC2008303F
:1025B000A900831634088312A400A501DB30B00003
:1025C000B1018A01BF210130A300F4308A01462203
:1025D0008A150A163525640083164708003C8A11BF
:1025E0000A16831203193F2B640083164708013C27
:1025F0008A110A168312031D062B83160301B41ECB
:10260000013E0319B412031DB4168312640083162D
:102610004708023C8A110A168312031D182B8316E1
:102620000301B41F013E0319B413031DB417831231
:10263000640083164708033C8A110A168312031D9F
:102640002A2B83160301341F013E03193413031D83
:1026500034178312640083164708043C8A110A1653
:102660008312031D3C2B83160301341E013E031904
:102670003412031D341683128A110A16A32A8316F4
:10268000510883128A01DC208316500883128A01C4
:10269000DC2055308A01DC203D308A01DC203330DB
:1026A0008A01DC2030308A01DC202D308A01DC20D8
:1026B00036308A01DC2030308A01DC2020308A016B
:1026C000DC2044308A01DC203D308A01DC203530BA
:1026D0008A01DC2030308A01DC202D308A01DC20A8
:1026E00037308A01DC2030308A01DC208316510823
:1026F00083128A01DC208316490883128A01DC20B8
:102700004C308A01DC203D308A01DC2045308A01D2
:10271000DC2067308A01DC2072308A01DC20203026
:102720008A01DC2052308A01DC203D308A01DC2025
:1027300053308A01DC206C308A01DC2065308A014C
:10274000DC2065308A01DC2070308A01DC20033017
:10275000A300E8308A0146220130A300F4308A0148
:1027600046228A150A163525640083164708003C60
:102770008A110A1283120319C82B640083164708B2
:10278000013C8A110A168312031DCF2B83161E30BB
:10279000DF003C30BA0083128A110A16FA2B64005B
:1027A00083164708023C8A110A12831203198F2CE0
:1027B000640083164708033C8A110A168312031D1E
:1027C000EA2B83163230DF004630BA0083128A11BA
:1027D0000A16FA2B640083164708043C8A110A166D
:1027E00083120319112D87128316871283128A11FF
:1027F0000A16AC2B8316510883128A01DC2083163B
:102800004A0883128A01DC2083165F0883128A013A
:10281000BB202D308A01DC2083163A0883128A01FE
:10282000BB2020308A01DC206D308A01DC20703032
:102830008A01DC2068308A01DC205830F6009E30A6
:10284000F7008316DE01E4018312101076088E0073
:1028500077088F000C108A150A1635256400831638
:102860004708003C8A110A16831203193F2B83166E
:10287000D130C60005308312B6001030B4004C30A1
:10288000AA004030AB00AE01AF0168308A0176216A
:102890006A308A017621F1308A01762101308A017D
:1028A00076210D308A0176218316460883128A012B
:1028B00076210530B6000830B4004C30AA00AB01D8
:1028C0006430AC00AD010730A9002030B000013009
:1028D000B100A50138308A0162218A110A16031C51
:1028E000712C3D088316DD005D088312A600A70148
:1028F0004530A2001830A3008A01C1228316DD00F2
:1029000083122730A30010308A0197228316DD003E
:10291000510883128A01DC2083164B0883128A0136
:10292000DC2053308A01DC2070308A01DC206530E5
:102930008A01DC2065308A01DC2064308A01DC20D9
:1029400020308A01DC2083165D0883128A01BB20B7
:1029500020308A01DC2054308A01DC2069308A0171
:10296000DC206D308A01DC2065308A01DC202030DB
:102970008A01DC2083165E0883128A01BB202E3078
:102980008A01DC208316640883128A01BB20203070
:102990008A01DC20640083165F085D028A110A1632
:1029A0008312031C2B2C1014640083163A085D025A
:1029B0008A110A1683120318AC2B64008A110A16B6
:1029C0000C1CDD2C2030870683168712E40A640075
:1029D00064080A3C8A110A168312031DF32C83161D
:1029E000E401DE0A831210100F088316A30083127D
:1029F0000E088316A200831276088316A20783129C
:102A000077080318013E8316A307230883128F005B
:102A10008316220883128E000C1010148A110A16D5
:102A20002B2C8316510883128A01DC2083164A0856
:102A300083128A01DC2045308A01DC2067308A015C
:102A4000DC2072308A01DC2020308A01DC20543006
:102A50008A01DC2065308A01DC2073308A01DC20A9
:102A600074308A01DC2069308A01DC206E308A01F2
:102A7000DC2067308A01DC200330A300E8308A01C3
:102A80004622051683160512473083128A01452215
:102A9000051283160512F53083128A01452205308E
:102AA000B6001030B4004C30AA004030AB00AE018C
:102AB000AF0168308A0176216A308A017621F530CB
:102AC0008A017621AF308A017621BF308A017621D2
:102AD000B3308A017621B2308A017621C1308A0171
:102AE0007621DB308A017621B3308A017621E93004
:102AF0008A01762196308A0145228A150A163525E3
:102B0000640083164708003C8A110A1683120319D1
:102B10003F2B0530B6001030B4004C30AA004030D6
:102B2000AB00AE01AF0120308A01762105308A0169
:102B300076211B308A01762102308A017621BE304F
:102B40008A0176210530B6000830B4004C30AA0066
:102B5000AB016430AC00AD010430A9002030B000FE
:102B60000130B100A50138308A0162218A110A16AC
:102B7000031CBA2D3A088316B900510883128A0142
:102B8000DC2083164B0883128A01DC2045308A0141
:102B9000DC2067308A01DC2072308A01DC202030A2
:102BA0008A01DC208316390883128A01BB20203079
:102BB0008A01DC2020308A01DC200730B60040305A
:102BC000B4005430AA004030AB00AE01AF01443035
:102BD0008A01762141308A01762154308A0176219A
:102BE00041308A0176212C308A01762154308A01C5
:102BF000762149308A0176214D308A01762145308F
:102C00008A0176212C308A017621A90183163908A0
:102C10008312A400A5017530B0000130B1008A0113
:102C2000E2210D308A0176218A110A167D2D831644
:102C3000510883128A01DC208316500883128A010E
:102C4000DC2054308A01DC2069308A01DC206D30C0
:102C50008A01DC2065308A01DC202C308A01DC20EE
:102C600020308A01DC2041308A01DC2068308A0172
:102C7000DC2020308A01DC2026308A01DC20203054
:102C80008A01DC2057308A01DC2068308A01DC2090
:102C90000330A300E8308A0146228A150A1635253A
:102CA000640083164708003C8A110A128312031934
:102CB000C82B640083164708013C8A110A16831248
:102CC000031D6E2E8316E4018312EC01ED018316C1
:102CD000D801DE0183128A110A16172E64008316AA
:102CE0004708023C8A110A168312031D942E0530F0
:102CF0008316B8076400FB3038028A110A16831263
:102D0000031C862E8316FF30B80083128316380802
:102D10008312A800F430A2000130A30001308A0120
:102D200002207D308A014522640083164708033C57
:102D30008A110A168312031DB22EE801E901E60189
:102D4000E701E401E501EA01EB018316A401A50115
:102D5000A601A701A801A901AA01AB0183128A114A
:102D60000A16172E640083164708043C8A110A16B7
:102D70008312031DD72E05308316B8026400053078
:102D800038028A110A1683120318C92E8316B80155
:102D90008312831638088312A800F430A200013091
:102DA000A30001308A0102207D308A01452283166A
:102DB000510883128A01DC208316490883128A0194
:102DC000DC2054308A01DC2069308A01DC206D303F
:102DD0008A01DC2065308A01DC2020308A01DC2079
:102DE0006D08A5006C088A01BC203A308A01DC20FD
:102DF00064000A30831658028A110A1683120318D7
:102E0000042F30308A01DC208316580883128A018F
:102E1000BB203A308A01DC2064000A3083165E024F
:102E20008A110A1683120318182F30308A01DC2009
:102E300083165E0883128A01BB2083165108831211
:102E40008A01DC2083164A0883128A01DC20413083
:102E50008A01DC2068308A01DC2020308A01DC20F5
:102E60002B308A01DC206608A0006708A1006430CE
:102E7000A200A3018A01A522FE002108FF007F080D
:102E8000A5007E088A01BC202E308A01DC2066085D
:102E9000A0006708A1006430A200A3018A01A52256
:102EA00024088316BE0064000A303E028A110A1606
:102EB000831203185E2F30308A01DC2083163E080F
:102EC00083128A01BB2020308A01DC202D308A0148
:102ED000DC206808A0006908A1006430A200A301FA
:102EE0008A01A522FE002108FF007F08A5007E08B8
:102EF0008A01BC202E308A01DC206808A000690805
:102F0000A1006430A200A3018A01A522240883162F
:102F1000BE0064000A303E028A110A1683120318AA
:102F2000942F30308A01DC2083163E0883128A01F8
:102F3000BB208316510883128A01DC2083164B08BC
:102F400083128A01DC2057308A01DC2068308A0134
:102F5000DC2020308A01DC202B308A01DC20831623
:102F600025088312A5008316240883128A01BC2039
:102F700020308A01DC202D308A01DC2083162708CE
:102F80008312A5008316260883128A01BC208A11A9
:102F90000A164D2E8316510883128A01DC208316EF
:102FA000500883128A01DC204F308A01DC20623015
:102FB0008A01DC2064308A01DC2069308A01DC204F
:102FC00069308A01DC2020308A01DC2043308A010C
:102FD000DC206C308A01DC2072308A01DC20443035
:102FE0008A01DC2074308A01DC2063308A01DC2015
:102FF0003D308A01DC2044308A01DC2020308A0107
:10300000DC200330A300E8308A0146228A150A1624
:103010003525640083164708003C8A110A12831282
:103020000319C82B640083164708033C8A150A1647
:103030008312031D37280530B6001030B4004C3021
:10304000AA004030AB00AE01AF0168308A017621A2
:103050006A308A017621F1308A01762104308A01B2
:103060007621C7308A0176218A110A16CA2F0530C7
:10307000B6001030B4004C30AA004030AB00AE01B6
:10308000AF0168308A0176216A308A017621F130F9
:103090008A01762103308A017621C6308A017621A1
:1030A0000530B6000830B4004C30AA00AB01C8307F
:1030B000AC00AD010B30A9002030B0000130B100F0
:1030C000A50138308A0162218A150A16031C682876
:1030D00064003B08433C8A150A160319B928831675
:1030E000510883128A01DC208316500883128A015A
:1030F000DC204E308A01DC206F308A01DC20203059
:103100008A01DC2044308A01DC2054308A01DC2032
:1031100043308A01DC2020308A01DC2043308A01E0
:10312000DC206F308A01DC2064308A01DC206530CD
:103130008A01DC2073308A01DC2020308A01DC2007
:1031400053308A01DC2065308A01DC2074308A012A
:10315000DC2020308A01DC203A308A01DC20293052
:103160008A01DC200730A300D0308A0146228A0180
:10317000C82B8316510883128A01DC208316490864
:1031800083128A01DC2083160430C0000530D3008E
:1031900083128A150A16E12083160630C000073014
:1031A000D30083128A150A16E12083160830C00066
:1031B0000930D30083128A150A16E1208A150A16EF
:1031C000062883164008383E840083120008FE005B
:1031D000C0307E05FE00FF017E08A0007F08A10030
:1031E00006308A016E228316BE003E08033C8A1513
:1031F0000A168312031C10298A150A160321CC0013
:103200008A150A16102919308A0083163E0883127F
:103210000C3E03188A0A82002034133412342534F9
:1032200083164008383E840083120008FE003030C8
:103230007E05CD004D08A000A10104308A016E2258
:10324000CD0083164008383E840083120008FE003B
:103250000F307E05CE0083165308383E840083125B
:103260000008FE00F0307E05CF004F08A000A1014D
:1032700004308A016E22CF0083165308383E840042
:1032800083120008FE000F307E05D0008316BE01B9
:1032900083126400053083163E028A150A168312D3
:1032A0000318682983163E084C3E840083120008E8
:1032B000FE0030307E07FE00FF01FF0D7E088A0110
:1032C000DC208316BE0A8A150A168312031D4929BB
:1032D00020308A01DC2008008316510883128A01FD
:1032E000DC208316500883128A01DC2049308A01D1
:1032F000DC206D308A01DC2061308A01DC20203046
:103300008A01DC2044308A01DC2069308A01DC201B
:1033100073308A01DC2044308A01DC2074308A0159
:10332000DC2063308A01DC203D308A01DC2055300E
:103330008A01DC2020308A01DC2043308A01DC2035
:103340006C308A01DC2044308A01DC2074308A0130
:10335000DC2063308A01DC203D308A01DC204430EF
:103360008A01DC208316510883128A01DC2083162F
:10337000490883128A01DC2053308A01DC206F3037
:103380008A01DC2063308A01DC203D308A01DC20A8
:1033900052308A01DC2020308A01DC2046308A014C
:1033A000DC2061308A01DC206E308A01DC203D3077
:1033B0008A01DC204C308A01DC2020308A01DC20AC
:1033C00045308A01DC2078308A01DC2069308A01AE
:1033D000DC2074308A01DC203D308A01DC20503052
:1033E0008A01DC200330A300E8308A0146228A15D6
:1033F0000A1635250130A300F4308A014622640004
:1034000083164708003C8A110A1283120319C82B3D
:10341000640083164708013C8A150A1683120319B3
:10342000482A640083164708023C8A150A1683124C
:103430000319F52A640083164708033C8A150A1607
:103440008312031D3C2A0530B6000430B40054300A
:10345000AA004030AB00AE01AF01E4308A01762112
:1034600005308A01762101308A01762103308A01F4
:10347000762113308A017621640083164708043CC4
:103480008A150A1683120319102C8A150A16F729B1
:103490008316510883128A01DC2083165008831298
:1034A0008A01DC2083160F30B5004030C500103093
:1034B000DC0083128A150A16762283160F30B500B7
:1034C0005030C5001030DC0083128A150A167622AF
:1034D00083160730B5006030C5000830DC00831269
:1034E0008A150A1676228A150A16F729EC308316F1
:1034F00045078312FE00FF01FF0D7E0883165C075F
:10350000BF003F08003CBF0005308312B600043006
:10351000B4005430AA004030AB00AE01AF01E4303B
:103520008A01762106308A01762102308A017621CD
:103530008316450883128A01762183165C0883125C
:103540008A01762183163F0883128A01762105308D
:10355000B6000230B4005430AA00AB019630AC0083
:10356000AD010330A9002030B0000130B1008A0164
:1035700059218A150A16031CCD2A83165C0883126A
:10358000A9002030B0000130B100A50138308A0117
:1035900062218A150A16031CCD2A8316BE018312E6
:1035A000640083163E0835028A150A168312031C2E
:1035B000F12A0230A90083163E08383E84008312A7
:1035C0000008FE007E08A400A501DB30B000B101B8
:1035D0008A01CF218316BE0A8A150A168312031D9B
:1035E000D02A64308A0145220800831651088312CC
:1035F0008A01DC208316500883128A01DC205330B4
:103600008A01DC206F308A01DC2063308A01DC20F3
:1036100020308A01DC2025308A01DC2020308A011C
:10362000DC2048308A01DC2069308A01DC203D3012
:103630008A01DC2055308A01DC2020308A01DC2020
:103640004D308A01DC2065308A01DC203D308A0162
:10365000DC204C308A01DC2020308A01DC204C3018
:103660008A01DC206F308A01DC203D308A01DC20B9
:1036700044308A01DC200330A300E8308A0146226E
:103680000530B6000430B4005430AA004030AB001E
:10369000AE01AF01E4308A01762106308A0176213D
:1036A00002308A01762110308A01762102308A01A7
:1036B000762102308A0176210530B6000230B4004E
:1036C0005430AA00AB016430AC00AD010630A90053
:1036D0002030B0000130B100A50138308A016221EC
:1036E0008A150A16031C742B3B08FB003C08FA00E1
:1036F0008316510883128A01DC208316490883123D
:103700008A01DC2050308A01DC203D308A01DC2037
:1037100049308A01DC206D308A01DC2061308A0169
:10372000DC2020308A01DC2020308A01DC2053306C
:103730008A01DC206F308A01DC2063308A01DC20C2
:1037400020308A01DC207A08A0007B08A1000A3022
:10375000A200A3018A01A522FE002108FF007F0824
:10376000A5007E088A01BC202E308A01DC207A0860
:10377000A0007B08A1000A30A200A3018A01A522B3
:103780002408FE002508FF007F08A5007E088A01A6
:10379000BC2020308A01DC208A150A16352501302C
:1037A000A300F4308A014622640083164708003CD7
:1037B0008A150A16831203196C29640083164708B8
:1037C000013C8A150A168312031DED2B831609305E
:1037D000BE0083128A150A160C256400831647085A
:1037E000043C8A150A168312031DFD2B831608302C
:1037F000BE0083128A150A160C256400831647083A
:10380000033C8A150A168312031D0D2C83160730FC
:10381000BE0083128A150A160C258A150A16402B3B
:103820008316510883128A01DC2083165008831204
:103830008A01DC2046308A01DC2061308A01DC20EC
:103840006E308A01DC2020308A01DC2048308A0179
:10385000DC2069308A01DC203D308A01DC204430E4
:103860008A01DC2020308A01DC204C308A01DC20F7
:103870006F308A01DC203D308A01DC204C308A0127
:10388000DC2020308A01DC204F308A01DC206630C9
:103890008A01DC2066308A01DC203D308A01DC2090
:1038A00055308A01DC200330A300E8308A0146222B
:1038B0000530B6000430B4005430AA004030AB00EC
:1038C000AE01AF01E4308A01762106308A0176210B
:1038D00002308A01762127308A01762102308A015E
:1038E0007621EB308A0176210530B6000230B40033
:1038F0005430AA00AB016430AC00AD010630A90021
:103900002030B0000130B100A50138308A016221B9
:103910008A150A16031C8C2C8316510883128A01FF
:10392000DC208316490883128A01DC2050308A018A
:10393000DC203D308A01DC2049308A01DC206D30FA
:103940008A01DC2061308A01DC2020308A01DC2001
:1039500048308A01DC2065308A01DC2078308A0119
:10396000DC2020308A01DC200230A9003B08A400C2
:10397000A501DB30B000B1018A01CF210230A900DE
:103980003C08A400A501DB30B000B1018A01CF21C1
:103990008A150A1635250130A300F4308A01462223
:1039A000640083164708003C8A150A16831203191F
:1039B0006C29640083164708013C8A150A16831295
:1039C000031DE92C8316FF30BE0083128A150A16E8
:1039D0000C25640083164708033C8A150A168312D7
:1039E000031DF92C83160130BE0083128A150A16B6
:1039F0000C25640083164708043C8A150A168312B6
:103A0000031D092D83160230BE0083128A150A1683
:103A10000C258A150A16582CED3083163E07BF0078
:103A20003F08003CBF0005308312B6000430B400EC
:103A30005430AA004030AB00AE01AF01E4308A013F
:103A4000762105308A01762104308A017621831699
:103A50003E0883128A01762183163F0883128A0169
:103A6000762164308A014522080000308A01102244
:103A70008316BE000530C7006400EB303E028A1595
:103A80000A168312031C452D08006400EB308316D0
:103A90003E028A150A1683120318522D831602302D
:103AA000C70083126400C03083163E028A150A16CE
:103AB000831203185F2D83160130C7008312640040
:103AC000963083163E028A150A16831203186C2D4F
:103AD00083160430C700831264006B3083163E02E5
:103AE0008A150A1683120318792D83160330C7002E
:103AF00083126400403083163E028A150A16831230
:103B00000318852D8316C701831264008A150A16CF
:103B100083168310B41E831483128318932D851784
:103B20008316851383124B308A0145228513831631
:103B30008513831208008316C20107308312B60072
:103B40001030B4000730B7000830B50083164208C3
:103B500083128A0172208316430883128A0172201D
:103B60008A015920F2008A015720F3007208A6004A
:103B70007308A7000230A200A3018A01C122FE003F
:103B80002508FF00B330FE026A30031C013EFF022D
:103B90007E08A0007F08A1006430A200A3018A0172
:103BA000A522F2002108F30064008A150A16831684
:103BB00083103419831483128318FD2D7208A60014
:103BC0007308A7001230A200A3018A01C122FE00DF
:103BD0002508FF007E08A0007F08A1000A30A2008F
:103BE000A3018A01A522FE002108FF0020307E07E4
:103BF000F2007F080318013EF300080064008316FA
:103C000062082D3C8A150A168312031D2A2E83167C
:103C100061088312A600A7011230A200A3018A0145
:103C2000C122FE002508FF007E08A0007F08A10039
:103C30000A30A200A3018A01A522FE002108FF008C
:103C40007E08203C8316E1002B30E20083128A15A7
:103C50000A16482E831661088312A600A7011230A7
:103C6000A200A3018A01C122FE002508FF007E08F0
:103C7000A0007F08A1000A30A200A3018A01A522AA
:103C8000FE002108FF0020307E078316E10083122A
:023C900008002A
:02400E00D420BC
:02401000FF3E71
:0443DC0004000500D4
:1043E0000F00150015000B0010001200FE00010068
:1043F0008000C0009400D4008A00CA009E00DE0045
:00000001FF
